:0E00020008308A0030290000FF00030E830141
:10001000A1007F08A0000A08A8008A01A00E040819
:10002000A2007708A3007808A4007908A5007A0840
:10003000A6007B08A700831383128C308400801EE7
:1000400023288C1A3628220884002308F700240865
:10005000F8002508F9002608FA002708FB00280800
:100060008A00210E8300FF0E7F0E09008A115C2892
:100070008C1E38281808AA001A08F800AA1C422862
:100080001812181600008A11632883166508F801F3
:10009000640203184E286408F7005A28F701083054
:1000A000E600E40DF70D650877020318F700F80D78
:1000B000E60B512883120034303062078400831627
:1000C000E3008312382883166308840078088000D0
:1000D000831262088316E1000130831262078316DF
:1000E000E300E4003230E500831245207708E200A7
:1000F00063086202031D8028831661088312E200F0
:100100008C128A11232883160617861783128A15E4
:100110008C29A1308400000803199B280230F800C4
:10012000F701F70B9128F80B90289730F700F70BA1
:100130009728800B8E2800346308620203199C28DC
:1001400030306307840000088316AC00013083124E
:1001500063078316AE008312A9018B1BA9178B13AB
:1001600083162E08E4003230E50083124520A91BD7
:100170008B177708E30083162C08F80083120034ED
:1001800083165C08DE005B08DF005D08003C031896
:10019000D5285F0884005E080002031DD2285F088E
:1001A000F800D728DF0ADD03C5280030F8008312E5
:1001B000003410308316DF00F701FA01DC0CDB0C91
:1001C000031CE8285D08F7070318FA0A5E08FA0717
:1001D000FA0CF70CF90CF80CDF0BDE288312003454
:1001E0008316A101AA01AA0183129C207808831614
:1001F000A1002008210203190929A2302A0784003E
:1002000021088000AA0A83129C2078088316A10086
:10021000F928A2302A0784008001A230AC002B0804
:10022000AD000A30AE00B201B3013030B50031305C
:10023000B6003230B7003330B8003430B900353052
:10024000BA003630BB003730BC003830BD00393022
:10025000BE006130BF006230C0006330C100643056
:10026000C2006530C3006630C4006730C500683026
:10027000C6006930C7006A30C8006B30C9006C30F6
:10028000CA006D30CB006E30CC006F30CD007030C6
:10029000CE007130CF007330D0007430D100753093
:1002A000D2007630D3007730D4007830D500793062
:1002B000D6007A30D700D8012C08AF002F08840070
:1002C0000008203C031D6629AF0A5E292F08840020
:1002D00000082D3C031972292F08840000082B3CCC
:1002E000031D77292F08AF0A8400000878292B30D6
:1002F000B40034082D3C031D8829AD080319842956
:100300002D0884002C0880000030F800F900882AAD
:10031000AE1B93292E0B8D299329AE1B9F292E08E6
:10032000243C03189F29AD0803199A292D0884003D
:100330002C0880000030F800F900882A052AAE0851
:100340000319DC292E08103C031DBC292F0884004A
:100350000008303C031DBC2901302F078400000831
:10036000783C0319BA2901302F0784000008583C53
:10037000031DBC290230AF072E08083C031DC82905
:100380002F0884000008303C031DC8290130AF0746
:100390002E08023C031DDB292F0884000008303C96
:1003A000031DDB2901302F0784000008623C031D78
:1003B000DB290230AF07052A2F0884000008303CF3
:1003C0000319E5290A30AE00052A01302F07840001
:1003D0000008783C0319F32901302F078400000836
:1003E000583C031DF8291030AE000230AF07052A33
:1003F00001302F0784000008623C031D032A0230ED
:10040000AE00AF07052A0830AE002F08B0002F0855
:1004100084000008303C031D0F2AAF0A072A2F086A
:1004200084000008D900403C03181D2A59085A3C92
:10043000031C1D2A590820381E2A5908DA00B53035
:10044000DB005908DC002E08DD008312C02078088C
:100450008316B100B10803196E2AFA012E08F700BD
:10046000AE1BFA03D9007A08DA003308DC00320840
:10047000DB005A08DE005908DD008312D920790814
:100480008316DB007808DA00B5303102FA015A072A
:10049000F8005B0803185B0FFA077808B2007A08C7
:1004A000B300AF0A2F0884000008D900403C0318AD
:1004B000602A59085A3C031C602A59082038612ACE
:1004C0005908DA00B530DB005908DC002E08DD00E1
:1004D0008312C02078088316B1002A2A2F08300220
:1004E000031D7D2AAD080319792A2D0884002C08E4
:1004F00080000030F800F900882AAD080319842A2A
:100500002D0884002F0880003208F8003308F90015
:100510007908831200340830F80000000000061348
:10052000831606130000B00D83128613031C9B2A4A
:100530008316861783120318A02A83168613831244
:10054000831606178312061BA72A8316A22AF80B06
:100550008D2A00000613831606130000861700007C
:10056000000006178312061BB72A8316B22AF80169
:100570000000861B78140613831606138312861355
:10058000831686138312003483168617000006171D
:10059000000083128613831686130000831206134D
:1005A000831606130310210DA038A800003024186C
:1005B0000130F700F70DF70DF70DF830F705770864
:1005C0002804AA00B00083128B2283162308A900F6
:1005D0002408AA002508AB00AC012308B000831250
:1005E0008B2283162208B00083128B2283162608E2
:1005F000B00083128B228316861300000617831225
:10060000061B042B8316FF2A0000000000000000D8
:100610008316861700008617000006170000831255
:10062000861383168613000083120613831606139F
:100630000310210DA038A800003024180130F70065
:10064000F70DF70DF70DF830F70577082804AA0025
:10065000B00083128B2278087818322B831627106B
:10066000342B831283162714271C642B8617000053
:10067000061700008312061B3F2B83163A2B8613A6
:1006800083168613000083120613831606130310C5
:10069000210DA038A800003024180130F700F70D14
:1006A000F70DF70DF830F70577082804AA00B00019
:1006B00083128B2278087818612B83162710632BFE
:1006C000831283162714342B8312003408308316C8
:1006D000AC007708AD008617000006178312061BD2
:1006E000732B83166E2B861B0314861F0310F80DC5
:1006F000000083160613831206138316AC0B6B2BB4
:10070000861700008312861383162D08031D861397
:10071000000006178312061B8F2B83168A2B0000FE
:10072000061383160613000083128613831686139E
:1007300083128A11F82B8316861700000617000013
:100740008312061BA52B8316A02B861383168613F4
:10075000000083120613831606130310250DA0381C
:10076000AB00003028180130F700F70DF70DF70D3A
:10077000F830F70577082B04AD00B00083128B2208
:1007800083162708AC002808AD002908AE00AF0189
:100790002708B00083128B2283162608B00083122C
:1007A0008B22831686170000061700008312061B93
:1007B000DB2B8316D62B8613831686130000831239
:1007C0000613831606130310250DA138AB00003065
:1007D00028180130F700F70DF70DF70DF830F70581
:1007E00077082B04AD00B00083128B22F701662B33
:1007F00078088316AA008613000006178312061BCA
:10080000032C8316FE2B000000000000000083165E
:10081000861700002A08F80083120034F801F90155
:10082000F701FA0183163108031D192C300803194A
:10083000332C1030B2000310AE0DAF0DF70DFA0DD2
:1008400031087A02031D262C30087702031C2F2C56
:100850003008F702031CFA033108FA020314F80DFA
:10086000F90DB20B1B2C000083128A11F42E8E306E
:10087000F70083163308F8003208F900FA01F80887
:10088000031D4C2C7908F800F9010830F702F8082C
:10089000031D4C2CF701542C0310F81B532CF90D9D
:1008A000F80DF7034C2CF81300008312003480304D
:1008B000831C5D2C8316BB0683128316C001C10105
:1008C0003708BF003B08BF0636080319482DBE0095
:1008D000F7003A080319512DBE020319EE2C031C30
:1008E000AD2C3B08C400C4173C08C3003D08C2003F
:1008F000C1010310C40CC30CC20CC10CBE0B782C7C
:10090000BF1F852C4014652D40103E104016B93095
:1009100084007A2D4012BF1B972C3E1CA22CC40CC5
:10092000C30CC20CC10CF70A0319602DA22CC41B06
:10093000A52C0310C10DC20DC30DC40DF70303197F
:10094000602D972C40170D2D40133708BF00B71F9F
:10095000AB2CC417592DC413592D3A08BE00F7000B
:100960003608BE023708C400C4173808C300390867
:10097000C200C1010310C40CC30CC20CC10CBE0BDD
:10098000B92CBF1FC62CC014652DC0103E10C01658
:10099000BD3084007A2DC012BF1BD82C3E1CE32C26
:1009A000C40CC30CC20CC10CF70A0319602DE32C54
:1009B000C41BE62C0310C10DC20DC30DC40DF703FB
:1009C0000319602DD82CC0170D2DC0133B08BF0094
:1009D000BB1FEC2CC417592DC413592D3B08C40060
:1009E000C4173C08C3003D08C200BF1FFB2CC41342
:1009F0004015652D4011C1013E10B93084007A2D9B
:100A0000BF1B232D3708BF003E1C0D2DC40CC30C8B
:100A1000C20CC10CF70A0319602DC11F1E2DC20A9A
:100A2000031D1E2DC30A031D1E2DC40A031D1E2DEA
:100A3000C40CC30CC20CF70A0319602D401BA42C74
:100A4000C01BE52C422D8030C406C41F2B2D652D04
:100A50003B08BF00382D3708BF00C408031D382DE0
:100A6000C308031D382DC208031D382DF701592D69
:100A7000C41B422D0310C10DC20DC30DC40DF70BD5
:100A8000382D602DBF1F462DC417592DC413592D65
:100A90003A08F7003B08C4003C08C3003D08C20008
:100AA000592D3608F7003708C4003808C300390844
:100AB000C2004408F8004308F9004208FA00982DE3
:100AC000F701F801F901FA01982DC101C209C30922
:100AD000C409C109C10A031D732DC20A031D732D68
:100AE000C30A0319C40A4018842CC018C52C401925
:100AF000FA2C282D0008C207031C842DC30A031DED
:100B0000842DC40A03193E1484030008C307031C80
:100B10008C2DC40A03193E1484030008801F803AF8
:100B2000C40703183E14401A8A2CC01ACB2C002D7F
:100B30000000831200348316320803190C2EBA0009
:100B4000360803190C2EBA070318AD2D7F30BA02F0
:100B5000031C0C2E03190C2EB12D8130BA0703187B
:100B60000C2E3A08F700F801F901FA013308BE002B
:100B7000BE173408BD003508BC001830BA00BB01F0
:100B80003C1CDA2D3908FA07031CCC2DF90A031D89
:100B9000CC2DF80A0319BB173808F907031CD32D0D
:100BA000F80A0319BB173708B400B4173408F8075C
:100BB0000318BB17BB0DF80CF90CFA0CBE0CBD0CDE
:100BC000BC0C0310BA0BBF2D0130F70703180C2E15
:100BD000F81BF12DBE0DFA0DF90DF80DF7030319F1
:100BE0000C2EBE1F022EFA0A031D022EF90A031D47
:100BF000022EF80A031D022EF80CF90CFA0CF70A63
:100C000003190C2E3308BB003708BB06BB1F0A2E86
:100C1000F817102EF813102EF701F801F901FA0158
:100C2000000083120034831636080319D92EC2003F
:100C30003A080319D92EC202031C232E7F30C207A3
:100C40000318D92E292E8130C202031CD92E031974
:100C5000D92E4208F700F801F901FA01C10137085D
:100C6000C000C0173808BF003908BE001930C200E4
:100C70003D08BE0203184C2E0130BF0203184C2E53
:100C8000C00203184C2EC10203184C2EC10AC00A20
:100C9000BF0A3D08BE077E2E3C08BF020318672E20
:100CA0000130C0020318672EC1020318672EC10A63
:100CB000C00A3C08BF073D08BE07031C7E2EBF0AC2
:100CC000031D7E2EC00A031D7E2EC10A7E2E3B0808
:100CD0008038C00203187D2E0130C10203187D2E1A
:100CE000C10A3B088038C0073C08BF07031C5B2EC5
:100CF000C00A031D5B2EC10A5B2E7A14C20B812E23
:100D00008C2E0310BE0DBF0DC00DC10D0310FA0DCA
:100D1000F90DF80DC30D382E431C942E0310F80C5A
:100D2000F90CFA0CC30C972EF7030319D92EC31B29
:100D3000C02E0310BE0DBF0DC00DC10D3D08BE027B
:100D40000318AC2E0130BF020318AC2EC0020318EA
:100D5000AC2EC102031CCF2E3C08BF020318B72ED5
:100D60000130C0020318B72EC102031CCF2E3B086E
:100D70008038C0020318C02E0130C102031CCF2EE0
:100D8000FA0A031DCF2EF90A031DCF2EF80A031D00
:100D9000CF2EF70A0319D92EF80CF90CFA0C3708E4
:100DA000C2003B08C206C21FD72EF817DD2EF8136B
:100DB000DD2EF701F801F901FA0100008312003479
:100DC0008316A401A501A601A701A801A901AA01F2
:100DD000AB01AC01AD012108AF002008AE00B101AC
:100DE0006430B00083120E2C79088316A5007808B1
:100DF000A4002108B3002008B2008312372477082A
:100E00008316AE007808AF007908B0007A08B10008
:100E10002508DC002408DB00DE016430DD008312DD
:100E2000D9207908FA0078088316B2007908B3004F
:100E300083123724831483163108B9003008B800B0
:100E40002F08B7002E08B6007A08BD007908BC004C
:100E50007808BB007708BA00831257247A088316F3
:100E6000A9007908A8007808A7007708A600230839
:100E7000B3002208B2008312372477088316AE002D
:100E80007808AF007908B0007A08B100B5003008E2
:100E9000B4002F08B3002E08B200B901B8017030B9
:100EA000B7008430B60083129B257A088316AD0004
:100EB0007908AC007808AB007708AA002D08B900C3
:100EC0002C08B8002B08B7002A08B600BD01403036
:100ED000BC001C30BB008C30BA00831213267A0889
:100EE0008316AD007908AC007808AB007708AA003B
:100EF0002908B9002808B8002708B7002608B60056
:100F0000BD01BC017030BB008430BA0083121326CF
:100F100077088316AE007808AF007908B0007A0829
:100F2000B1002508B3002408B200831237248310CF
:100F30007A088316B9007908B8007808B7007708EE
:100F4000B6003108BD003008BC002F08BB002E08D9
:100F5000BA008312572477088316B2007808B300CA
:100F60007908B4007A08B5002D08B9002C08B8003B
:100F70002B08B7002A08B600BD01BC016130BB00D8
:100F80008A30BA0083121326831083163508B900FD
:100F90003408B8003308B7003208B6007A08BD003C
:100FA0007908BC007808BB007708BA008312572480
:100FB000003483162B08B63CAB00FA012C08AF00B6
:100FC000AC170310AC0CAD0CAE0CFA0CF90CF80C11
:100FD000F70CAB0BE12FAF1FF82FF709F809F90950
:100FE000FA09F70A0319F80A0319F90A0319FA0AA0
:060FF00083128A1573282C
:10100000F701F801F901FA018316B301B401B50142
:10101000B6013208310430042F0403193F28203070
:10102000B7000310AB0DAC0DAD0DAE0DB30DB40D8F
:10103000B50DB60D32083602031D282831083502D9
:10104000031D282830083402031D28282F083302E6
:10105000031C39282F08B3023008031C300FB402D8
:101060003108031C310FB5023208031C320FB602DF
:101070000314F70DF80DF90DFA0DB70B1128000048
:10108000B33084008312003404088316A5002408BA
:10109000A600031968282308B5002208B400210817
:1010A000B3002008B200B901B8012030B700823087
:1010B000B6008A1183129B258A157A088316A3002D
:1010C0007908A2007808A1007708A000A60B4B2899
:1010D0002308AE002208AD002108AC002008AB00B8
:1010E0008A118312D92F8A157A088316A3007908EA
:1010F000A2007808A1007708A000A31F8C28A503F0
:10110000A516A009A109A209A309A00A0319A10A09
:101110000319A20A0319A30A3B30AA009A30A900B6
:10112000CA30A800A7010A30A60024080319A50A9E
:101130002308AE002208AD002108AC002008AB0057
:101140002A08B2002908B1002808B0002708AF001B
:101150008312002000088316A000840A0008A10062
:10116000840A0008A200840A0008A300FD30840756
:10117000F708031DCE28240A26020319CE282508C5
:101180000319D0280F3926020319C8280318142977
:10119000A51B1429251BD02820300B292030A5059C
:1011A000A51EE328A5122408031DA5037708A500A2
:1011B0002D3083120C1ADE288316D9289900831645
:1011C0002508F700A50124082602031DF628770844
:1011D000A5002E3083120C1AEF288316EA289900F6
:1011E00083162508F7002030A50500303030A51EF5
:1011F0000B29A5122408031DA5037708A5002D308F
:1012000083120C1A052983160029990083162508D4
:10121000F700A5013030F707770883120C1A12295E
:1012200083160D29990083162A08AE002908AD00FF
:101230002808AC002708AB00B201B101B0010A30A8
:10124000AF00831200207A088316AA007908A9004B
:101250007808A8007708A700A60B98288312003406
:1012600084011F308305703083168F001930990078
:101270002230980090308312980083161F129F121C
:101280001B0880399B0007309C008312AA01AB0128
:101290000130AC00AD01AE01AF01E201E301641029
:1012A000E410E501E601E701E801E901EA01EB01EB
:1012B000EC01ED01EE01EF01F001F101F2017030FE
:1012C00083168F001F129F121B0880399B00831208
:1012D0001F10073083169C0005080630F700F70B37
:1012E0006F2900001C0883120D1383160108C739EB
:1012F00008388100831290010030F800920000301D
:1013000083169200C03083128B0483168C1605124C
:10131000831205168A1183288A1532308316A1009C
:101320008A11831289208A15831605158312051DDB
:101330009B2964149C296410FA308316A1008A1139
:10134000831289208A156418F52B831605158312DC
:10135000051DA529E4108316051283120512E9085C
:10136000031DF42B6808013C031CF42B6A08243C81
:101370000319C0298A119C208A157808EA00B62929
:101380008A119C208A157808EA006A08473C031DE8
:10139000F32B8A119C208A157808EA006A08503CD1
:1013A000031DF32B8A119C208A157808EA006A082D
:1013B000523C031DF32B8A119C208A157808EA0001
:1013C0006A084D3C031DF32B8A119C208A1578086E
:1013D000EA006A08433C031DF32B8A119C208A15FE
:1013E0007808EA0083160510831205148A119C20E0
:1013F0008A157808EA006A082C3C0319052A8A1124
:101400009C208A157808EA00FB298A119C208A15FD
:101410007808EA006A08413C031D142AE414831684
:10142000051283120516152AE4108A119C208A15CC
:101430007808EA00E41CEB2B2E308316A0008A11FA
:101440008312F0208A157908EC007808EB006C080C
:101450008316A000A101831269088316A5008312D8
:1014600068088316A400831267088316A3008312FA
:1014700066088316A2002008A6008A118312C422DF
:101480008A150130E6070318E70A0319E80A031969
:10149000E90A6B088316A000A1018312690883166C
:1014A000A500831268088316A400831267088316B8
:1014B000A300831266088316A2002008A6008A11E2
:1014C0008312C4228A150130E6070318E70A0319BC
:1014D000E80A0319E90A2C308316A0008A11831246
:1014E000F0208A157908EE007808ED006E08831662
:1014F000A000A101831269088316A5008312680861
:101500008316A400831267088316A300831266085B
:101510008316A2002008A6008A118312C4228A150D
:101520000130E6070318E70A0319E80A0319E90A74
:101530006D088316A000A101831269088316A50017
:10154000831268088316A400831267088316A30019
:10155000831266088316A2002008A6008A1183124F
:10156000C4228A150130E6070318E70A0319E80ABE
:101570000319E90A8A119C208A157808EA00831663
:10158000A101831269088316A500831268088316D7
:10159000A400831267088316A300831266088316CB
:1015A000A20083126A088316A6008A118312C4223D
:1015B0008A150130E6070318E70A0319E80A031938
:1015C000E90A8A119C208A157808EA008316A1018D
:1015D000831269088316A500831268088316A40085
:1015E000831267088316A300831266088316A2007D
:1015F0002C30A6008A118312C4228A150130E60716
:101600000318E70A0319E80A0319E90A2E308316BA
:10161000A0008A118312F0208A157908EC0078085E
:10162000EB006C088316A000A101831269088316E1
:10163000A500831268088316A40083126708831626
:10164000A300831266088316A2002008A6008A1150
:101650008312C4228A150130E6070318E70A03192A
:10166000E80A0319E90A6B088316A000A101831296
:1016700069088316A500831268088316A4008312E4
:1016800067088316A300831266088316A200200849
:10169000A6008A118312C4228A150130E6070318B6
:1016A000E70A0319E80A0319E90A2C308316A00097
:1016B0008A118312F0208A157908EE007808ED006F
:1016C0006E088316A000A101831269088316A50085
:1016D000831268088316A400831267088316A30088
:1016E000831266088316A2002008A6008A118312BE
:1016F000C4228A150130E6070318E70A0319E80A2D
:101700000319E90A6D088316A000A1018312690874
:101710008316A500831268088316A4008312670845
:101720008316A300831266088316A2002008A60071
:101730008A118312C4228A150130E6070318E70ACA
:101740000319E80A0319E90A8A119C208A15780806
:10175000EA008316A101831269088316A50083128B
:1017600068088316A400831267088316A3008312F7
:1017700066088316A20083126A088316A6008A11DF
:101780008312C4228A150130E6070318E70A0319F9
:10179000E80A0319E90A8316A1018312690883166E
:1017A000A500831268088316A400831267088316B5
:1017B000A300831266088316A2000D30A6008A11CA
:1017C0008312C4228A150130E6070318E70A0319B9
:1017D000E80A0319E90A8316051283120512831613
:1017E000051083120510AF296E2E83160512831281
:1017F0000512E908031D6A2E6808013C031C6A2EC5
:10180000831605100130831285068316A501831205
:1018100069088316A900831268088316A80083123A
:1018200067088316A700831266088316A6008A112C
:1018300083129B238A1578088316A0000130831237
:1018400066078316A100831267088316A200003082
:1018500003180130A207831268088316A300003022
:1018600003180130A307831269088316A40000300F
:1018700003180130A407A5012408A9002308A80023
:101880002208A7002108A6008A1183129B238A152B
:1018900078088316A20020088312EC008316220821
:1018A0008312EB000130E6070318E70A0319E80A80
:1018B0000319E90A0130E6070318E70A0319E80AE1
:1018C0000319E90A8316A501831269088316A90082
:1018D000831268088316A800831267088316A7007E
:1018E000831266088316A6008A1183129B238A1529
:1018F00078088316A0000130831266078316A100C2
:10190000831267088316A200003003180130A20773
:10191000831268088316A300003003180130A30760
:10192000831269088316A400003003180130A4074D
:10193000A5012408A9002308A8002208A70021085F
:10194000A6008A1183129B238A1578088316A200A9
:1019500020088312EE00831622088312ED00013066
:10196000E6070318E70A0319E80A0319E90A013030
:10197000E6070318E70A0319E80A0319E90A6C08DD
:101980008316A10083126B088316A00083126E08D1
:101990008316A30083126D088316A2008A11831296
:1019A000E0268A157A08F2007908F1007808F0003C
:1019B0007708EF008316A501831269088316A90032
:1019C000831268088316A800831267088316A7008D
:1019D000831266088316A6008A1183129B238A1538
:1019E0007808E5000130E6070318E70A0319E80A5A
:1019F0000319E90A6508533C031D002D8030F006E9
:101A00008316A501831269088316A900831268084A
:101A10008316A800831267088316A700831266083E
:101A20008316A6008A1183129B238A157808E50085
:101A30000130E6070318E70A0319E80A0319E90A5F
:101A40008930840072088316A3007108A200700810
:101A5000A10083126F088316A0000630A400831231
:101A600044202C300C1E322D99008316A5018312C0
:101A700069088316A900831268088316A8008312D8
:101A800067088316A700831266088316A6008A11CA
:101A900083129B238A1578088316A00001308312D5
:101AA00066078316A100831267088316A200003020
:101AB00003180130A207831268088316A3000030C0
:101AC00003180130A307831269088316A4000030AD
:101AD00003180130A407A5012408A9002308A800C1
:101AE0002208A7002108A6008A1183129B238A15C9
:101AF00078088316A20020088312EC0083162208BF
:101B00008312EB000130E6070318E70A0319E80A1D
:101B10000319E90A0130E6070318E70A0319E80A7E
:101B20000319E90A8316A501831269088316A9001F
:101B3000831268088316A800831267088316A7001B
:101B4000831266088316A6008A1183129B238A15C6
:101B500078088316A0000130831266078316A1005F
:101B6000831267088316A200003003180130A20711
:101B7000831268088316A300003003180130A307FE
:101B8000831269088316A400003003180130A407EB
:101B9000A5012408A9002308A8002208A7002108FD
:101BA000A6008A1183129B238A1578088316A20047
:101BB00020088312EE00831622088312ED00013004
:101BC000E6070318E70A0319E80A0319E90A0130CE
:101BD000E6070318E70A0319E80A0319E90A6C087B
:101BE0008316A10083126B088316A00083126E086F
:101BF0008316A30083126D088316A2008A11831234
:101C0000E0268A157A08F2007908F1007808F000D9
:101C10007708EF008316A501831269088316A900CF
:101C2000831268088316A800831267088316A7002A
:101C3000831266088316A6008A1183129B238A15D5
:101C40007808E5000130E6070318E70A0319E80AF7
:101C50000319E90A6508573C031D302E8030F00651
:101C60008316A501831269088316A90083126808E8
:101C70008316A800831267088316A70083126608DC
:101C80008316A6008A1183129B238A157808E50023
:101C90000130E6070318E70A0319E80A0319E90AFD
:101CA0008930840072088316A3007108A2007008AE
:101CB000A10083126F088316A0000630A4008312CF
:101CC00044200D300C1E622E99000A300C1E662E28
:101CD0009900F92B8316051083120510831605123F
:101CE00010308312850602308316A000FA30A1005E
:101CF0008A11831289208A158316A00B762E8312EF
:041D00006E2E6300E0
:04400E00383FFF3FF9
:00000001FF
